:020000002728AF
:08000800882992002030D0216C
:100010000A289200120E0F3915200000D021120874
:100020000F3915200000D02108008A0182073034E2
:10003000313432343334343435343634373438347C
:1000400039344134423443344434453446340C303A
:1000500084008001840A841F292885018601831673
:10006000F0308500373086008312E22183160113B9
:100070008113811281110111011081148312013049
:10008000CA214030EA230230CA211E30DB21E72397
:100090002C30AB008B170B16A81F4C28A813AA0AEC
:1000A000E723061D8428861C712804218621A220AE
:1000B00086217C2158214030EA230C2186211921F8
:1000C000862181211430EA23F920862115218621F9
:1000D00072215430EA232E21862122218621772184
:1000E0004C282A218621AC204030EA23F5208621A5
:1000F00054211430EA232621862119215430EA2381
:100100006721862162214C282C308E0091204030BE
:10011000EA2391201430EA2391205430EA239120DD
:100120004C2805308D000E088E0A84000008861CBD
:100130009B2805209F2896009501392277228D0B58
:10014000932808000330CA212F086B290530960731
:1001500008000A30960708000430CA21950196016C
:10016000DA303002031CA920C7303002031CA9205A
:10017000B1303002031CA92098303002031CA920A2
:100180007E303002031CA92066303002031CA920F7
:100190005C303002031CA62051303002031CA62024
:1001A00048303002031CA62040303002031CA62039
:1001B00038303002031CA62032303002031CA62047
:1001C0002C303002031CA62027303002031CA6204E
:1001D00022303002031CA62019303002031CA92053
:1001E00015303002031CA9206D290530CA213108C1
:1001F0006B290630CA21320898005E3099008E22A1
:100200008A220A3096076D290730CA2133089800E0
:10021000193099008E226D290830CA2134089800BF
:10022000643099008E228A226D290930CA2135084E
:100230006B290A30CA2136089800463099008E2270
:1002400080226D290B30CA213E086B290C30CA214F
:100250003F086B290D30CA213B086B290E30CA219B
:100260000F309600C0303202031844290430960241
:1002700080303202031844290430960214303202CE
:1002800003184429043096026830330203185329B6
:100290009603483033020318532996031E30330265
:1002A0000318532996036C290F30CA213D086B2986
:1002B0003D082306031908003D08A300E72310307A
:1002C000CA2108001230CA212908A9016B2911305E
:1002D000CA212A086B2996009501392277222030FD
:1002E000D02108002030BA1B4330D0210800203034
:1002F000BA184C30D021080020303A1A4130D021B1
:1003000008002030AC1B4930D02108002030D02913
:10031000A000030EA1000408A20083128B1C9629E2
:100320008B101A3081000B118B16C3290B118B1205
:100330000330A700061CA3290000061C9829A70B60
:100340009C290310A929000006189829A70BA329A6
:100350000314A40D031CB429240FB4290930A500EB
:10036000A8172C30AB00C329A50BC3290930A50061
:100370002B0884002408A6002817A90A8000503002
:100380002B06031DAB0A22088400210E8300A00E59
:10039000200E09008D00FF30930000230800303844
:1003A0008F00CE2308004A30F523FF30F5238C035D
:1003B000031DD3290800940064308C00D321940BD2
:1003C000DC29080014308C00D32103308500861707
:1003D000861306308C00D3210330850086178613E0
:1003E00005308C00D3210330850086178613053035
:1003F0008C00D321023085008617861305308C00CF
:10040000D3210230850086178613083085008617B1
:10041000861305308C00D3210030850086178613A3
:10042000083085008617861305308C00D3210030F4
:1004300085008617861301308500861786130530E0
:100440008C00D32100308500861786130630850086
:100450008617861305308C00D3210030850086175F
:1004600086130C3085008617861305308C00D32147
:100470000800031010309100980199019A01960D1F
:10048000950D9A0D990D980D910B472A5C2A1A30FB
:1004900084005122193084005122183084005122E6
:1004A0003F2A033000079200921980003030000785
:1004B0009200921B800000341A089E000F39303ED3
:1004C0009F001E0E0F39303E9E0019089C000F3908
:1004D000303E9D001C0E0F390319702A303E712AE0
:1004E00020309C0018080F39303E9B0000341C0857
:1004F000D0211D08D0211E08D0211F08D021003492
:100500000430832A033092000310950C960C920B52
:10051000842A00341508960095010800950196017B
:100520000830910018080310990C03189507950CD2
:08053000960C910B942A003493
:1006000003308A000D0809238F00CE238F1F002B93
:100610000800820700001D2B362B452B4D2B552B38
:100620005D2B652B6D2B752B7D2B852B8D2B952BAA
:100630009D2BA52BAD2BBE2BC62B03308A00930A16
:10064000130882073134363430344234613475341F
:100650006434203441344C3444344C3420344434F5
:100660006934733470346C346134F93403308A0083
:10067000930A130882077634203431342E34303410
:10068000313420344A344E34A03403308A00930A83
:100690001308820749344134C33403308A00930A73
:1006A0001308820754344D34D03403308A00930A3F
:1006B0001308820753345034C43403308A00930A39
:1006C000130882074D344134D03403308A00930A32
:1006D0001308820752347034ED3403308A00930AD1
:1006E0001308820754345034D33403308A00930AF9
:1006F0001308820749346E34F43403308A00930AB5
:10070000130882074F343234A03403308A00930A2E
:100710001308820742344C34CD3403308A00930AE4
:10072000130882074F346334E33403308A00930A9A
:100730001308820742346134F43403308A00930A88
:100740001308820743346534EC3403308A00930A7B
:100750001308820750344134B33403308A00930ABB
:1007600013088207203420342034213420344B34C1
:100770006E346F3463346B342034A13403308A0018
:10078000930A130882074D347334E73403308A0028
:10079000930A1308820752347834E3340F0E073972
:1007A00085000617861786130F080F398500061770
:1007B000861786130613ED2B0F0E0F39850086174B
:1007C00086130F080F39850086178613EF2B01302B
:1007D0008F00DC2B80388F00DC2B1630F52B41305E
:1007E000F523FF30F523FF30F52B90009003031D18
:0407F000F62B0034B0
:02400E00F13F80
:00000001FF
